:10000000B201BC290408A20083160710831209302C
:10001000A30003101220A20CA30B0A280314122021
:100020000314B7290318172800000714192807100C
:1000300019280030A10062306029B216B21EB21237
:10004000B2192628B2155F2003184D280830A300E6
:100050007320A20DA30B2828B21E58207D207920E2
:10006000B21A4D20522022080310B729B216B21E30
:10007000B21232194028FE39B30032150310B729E5
:10008000321A4828A60032165F2003184D28260889
:10009000662003184D28B21EB72958207D20321142
:1000A0003212B211360884003408841780045E28A6
:1000B0003608840034098005841780050800522022
:1000C0007D20582079203308B2190138A200083069
:1000D000A300A20D03185220031C58207D20792074
:1000E000A30B692852207D203608840034080005BF
:1000F000FF3E3708840035095B283708840035083F
:1001000055282C08A0002D08A1000130A200A30151
:100110006400AF20031C9C28A20B8828FF30A30793
:1001200003188828A007031CA107031C08006430DB
:10013000A2000030A30088280221A8010830A300F3
:100140000321AF200318A80AAB1EA801A20CA30B21
:10015000A028AB1AA21303210314220808003608B2
:100160008400340884178004841300052B1B340694
:10017000FF3E0800A400290803140319B729B2217F
:10018000031C0800A00025188317240884002008F9
:1001900080008313A40AA903BB280408A60036081C
:1001A00084008030B3050830A70003100318B30A99
:1001B000E820A60CA70BD6280000AB1A330CE820C9
:1001C000BA210314E8202F08A3002E085321B729D1
:1001D0008413AB1FF728000834042B1F340680005B
:1001E000841700083404031C340680000329000827
:1001F0003404031C34062B1B340680008417340996
:100200008005032933172B081F39003EA1002A0857
:10021000043E0318A10A331F60293313A000031002
:10022000A10CA00C0310A10C200C6029A40029082B
:100230000319B7292518831724088400000883139D
:10024000B221A40AA9031829B31329080319B31763
:100250000530A8002730A30010303A210330A30056
:10026000E8303A21A30164303A21A3010A303A214F
:1002700024084129A2002508A1002408A0009621F5
:100280002008A000A8030319B313290803194B2958
:100290002802031808002008031DB313B31B08002D
:1002A000303EB229A301A200FF30A207031CA3071E
:1002B000031CB7290330A100E33060215429A101B8
:1002C000F43EA000A109FE30031C6929A007031811
:1002D0006629A0076400A10F662900002018702974
:1002E0002018722908000310A00DA10DFF3E03186D
:1002F00073292008B7290310A10CA00CFF3E031896
:100300007B292008B729A20004308629A8002308E9
:100310002102031D8D292208200204300318013018
:10032000031902302805031DFF30B729A501A401D8
:100330001030A600210DA40DA50D2208A40223084B
:10034000031C230FA5020318AC292208A4072308C5
:100350000318230FA5070310A00DA10DA60B9A29C2
:100360002008B729840031088A00300882008313EE
:100370000313831264000800831671308F00071185
:1003800005150710051485148516871105123030E0
:100390009F00063091008312051683160512831202
:1003A000E001E101DA01DB0156308A01032044302B
:1003B0008A01032072308A01032069308A010320F8
:1003C00076308A01032065308A01032032308A01A9
:1003D000032020308A01032053308A010320543047
:1003E0008A01032041308A01032052308A01032010
:1003F00054308A01032049308A0103204E308A019B
:10040000032047308A0103200D308A0103200A307F
:100410008A010320C8308A01522107168316071269
:1004200083120230A30058308A01532153308A01CD
:10043000032059308A0103204E308A0103204330C3
:100440008A01032048308A01032052308A010320A8
:100450004F308A0103204E308A01032049308A013F
:1004600003205A308A01032049308A0103204E308C
:100470008A01032047308A0103200D308A010320BE
:100480000A308A010320FA308A01522153308A014E
:10049000032065308A0103206E308A010320643016
:1004A0008A01032069308A0103206E308A0103200B
:1004B00067308A01032020308A01032045308A01F9
:1004C00003200D308A0103200A308A0103200730FF
:1004D000B6001030B4005430AA00AB01AE01AF0139
:1004E00045308A01CE200D308A01CE200730B6007B
:1004F0002030B4005430AA00AB016430AC00AD0130
:100500008A0181208A11031CAF2AE60053308A0138
:10051000032065308A0103206E308A010320743085
:100520008A01032020308A01032045308A010320FC
:100530003D308A01032020308A01032066088A01A9
:1005400003200D308A0103200A308A010320640051
:100550006608453C8A110319DE2A8A01432A4E3077
:100560008A0103206F308A01032020308A01032092
:1005700045308A01032020308A01032072308A012D
:10058000032065308A01032074308A01032075300E
:100590008A01032072308A0103206E308A01032011
:1005A00065308A01032064308A0103200D308A01FE
:1005B00003200A308A0103208A01432A53308A012A
:1005C000032065308A0103206E308A0103206430E5
:1005D0008A01032020308A01032053308A0103203E
:1005E00055308A01032044308A0103200D308A01EE
:1005F00003200A308A0103200730B6001030B4000F
:100600005430AA00AB01AE01AF0153308A01CE20B5
:1006100055308A01CE2044308A01CE200D308A0127
:10062000CE200730B6001030B4005430AA00AB0121
:10063000AE01AF0152308A01CE2044308A01CE2073
:1006400020308A01CE2064308A01CE2061308A01B8
:10065000CE2074308A01CE2065308A01CE202E3023
:100660008A01CE2074308A01CE2078308A01CE20D3
:1006700074308A01CE200D308A01CE200730B600BA
:100680002030B4005430AA00AB015830AC00023026
:10069000AD000E30A9008130B000B101A5013830A5
:1006A0008A01BA208A11031C142D64003808433CC7
:1006B0008A110319142D64308A01032061308A01E4
:1006C000032074308A01032065308A0103207330CF
:1006D0008A01032074308A01032072308A010320CA
:1006E00069308A0103206E308A01032067308A0155
:1006F00003203D308A01032020308A0103200E3080
:10070000A9000230B000B101A50138308A011621DC
:100710000D308A0103200A308A01032073308A01D8
:10072000032065308A01032074308A01032063307E
:100730008A0103206C308A0103206F308A01032074
:1007400063308A0103206B308A0103200D308A0157
:1007500003200A308A010320F001D0304507DC0075
:10076000FF300318013EDD00D0304407DE00FF30CB
:100770000318013EDF005E08A0005F08A1000430FE
:100780008A017621DE002108DF005C085E07EE00AA
:10079000D0304207DC00FF300318013EDD00D030CE
:1007A0004107DE00FF300318013EDF005E08A000B5
:1007B0005F08A10004308A017621DE002108DF00F5
:1007C0005C085E07ED00F101D0303F07DC00FF3030
:1007D0000318013EDD00D0303E07DE00FF30031875
:1007E000013EDF005E08A0005F08A10004308A011E
:1007F0007621DE002108DF005C085E07EC00D030C7
:100800003C07DC00FF300318013EDD00D0303B0721
:10081000DE00FF300318013EDF005E08A0005F0825
:10082000A10004308A017621DE002108DF005C0887
:100830005E07EF00D0303907DC00FF300318013EBF
:10084000DD00D0303807DE00FF300318013EDF0046
:100850005E08A0005F08A10004308A017621DE0056
:100860002108DF005C085E07F2001030EB00073063
:10087000B6000830B4000730B7000430B500D030FF
:100880008A01382000308A01382070088A01382017
:100890006E088A0138206D088A01382071088A01A3
:1008A00038206C088A0138206F088A0138207208C5
:1008B0008A0138206B088A01362064308A0152216F
:1008C0000730B6001030B4005430AA00AB01AE01BE
:1008D000AF0152308A01CE2045308A01CE204E3001
:1008E0008A01CE2020308A01CE2064308A01CE20B9
:1008F00061308A01CE2074308A01CE2065308A01B1
:10090000CE202E308A01CE2074308A01CE2078305D
:100910008A01CE2074308A01CE2020308A01CE2078
:100920006E308A01CE2064308A01CE2061308A0187
:10093000CE2074308A01CE2065308A01CE202E3040
:100940008A01CE2074308A01CE2078308A01CE20F0
:1009500074308A01CE200D308A01CE2072308A0197
:10096000032065308A0103206E308A010320613044
:100970008A0103206D308A01032065308A0103203B
:1009800020308A01032064308A01032061308A010B
:10099000032074308A01032065308A0103202E3041
:1009A0008A01032074308A01032078308A010320F1
:1009B00074308A01032020308A01032074308A01B8
:1009C00003206F308A01032020308A0103206E301B
:1009D0008A01032064308A01032061308A010320E8
:1009E00074308A01032065308A0103202E308A0189
:1009F000032074308A01032078308A010320743088
:100A00008A01032020308A0103200E30A900023021
:100A1000B000B101A50138308A0116210D308A01DC
:100A200003200A308A0103208A158B208A1557215A
:100A300064008A11851E2A2D8A153C220330A300EA
:100A4000E8308A01532105128316051264008312CF
:100A50008A01262D0330A30020308A0153218A11F8
:100A6000D6278A110D268A1137268A11612653301E
:100A70008A01032074308A01032065308A01032033
:100A800070308A01032020308A010320A9015A080E
:100A9000A4005B08A5000230B000B1018A01242146
:100AA00020308A01032046308A01032069308A0100
:100AB00003206C308A01032065308A0103203A301C
:100AC0008A01032020308A010320A9015208A400D2
:100AD000A5010230B000B1018A012421A901530807
:100AE000A400A5010230B000B1018A012421A901AE
:100AF0005408A400A5010230B000B1018A012421EC
:100B0000A9015508A400A5010230B000B1018A0175
:100B10002421A9015608A400A5010230B000B101AA
:100B20008A012421A9015708A400A5010230B000C0
:100B3000B1018A012421A9015808A400A5010230AD
:100B4000B000B1018A012421A9015908A400A5011E
:100B50000230B000B1018A0124212E308A01032025
:100B600063308A01032073308A01032076308A01C2
:100B700003200D308A0103200A308A0103205430FB
:100B80008A01032069308A0103206D308A01032025
:100B900065308A01032020308A010320A9016808FA
:100BA000A400A5010230B000B1018A012421A901ED
:100BB0006708A400A5010230B000B1018A01242118
:100BC0003A308A010320A9017B08A400A501023064
:100BD000B000B1018A012421A9017A08A400A5016D
:100BE0000230B000B1018A0124210D308A010320B6
:100BF0000A308A0103205A08A0005B08A1001C30BB
:100C0000A30021308A0183218A11031D182D8A1522
:100C10003C22DA01DB018A01142D05309F009F146C
:100C200064308A015F211E08E20041308A010320FE
:100C300044308A01032043308A01032031308A0185
:100C400003203D308A01032020308A010320A901BE
:100C50006208A400A5010230B000B1018A0124217C
:100C60000D308A0103200A308A0103200800093070
:100C70009F009F1464308A015F211E08E300413009
:100C80008A01032044308A01032043308A01032073
:100C900032308A0103203D308A01032020308A014E
:100CA0000320A9016308A400A5010230B000B1012E
:100CB0008A0124210D308A0103200A308A01032091
:100CC0000800DA0A0319DB0A57308A010320723060
:100CD0008A01032069308A01032074308A010320CD
:100CE00065308A01032020308A010320A901831680
:100CF00020088312A400A5010230B000B1018A01CE
:100D00002421A9017F08A400A5010230B000B1018F
:100D10008A012421A9016A08A400A5010230B000BB
:100D2000B1018A012421A9016908A400A5010230AA
:100D3000B000B1018A012421A9016508A400A50120
:100D40000230B000B1018A012421A9016408A40085
:100D5000A5010230B000B1018A012421A90168086F
:100D6000A400A5010230B000B1018A012421A9012B
:100D70006708A400A5010230B000B1018A01242156
:100D8000A9017B08A400A5010230B000B1018A01CD
:100D90002421A9017A08A400A5010230B000B10104
:100DA0008A012421A9017D08A400A5010230B00018
:100DB000B1018A012421A9017C08A400A501023007
:100DC000B000B1018A0124212C308A0103200330B4
:100DD000A9006208A400A5010230B000B1018A0197
:100DE00024212C308A0103200330A9006308A400C9
:100DF000A5010230B000B1018A0124210D308A0121
:100E000003200A308A0103200730B6001030B400F6
:100E10005430AA00AB01AE01AF0157308A01CE2099
:100E200052308A01CE2046308A01CE2020308A01FD
:100E3000CE2000308A01CE2000308A01CE20003042
:100E40008A01CE2015308A01CE200D308A01CE20B5
:100E5000A901831620088312A400A501CD30B0009B
:100E6000B1018A012421A9017F08A400A501CD3088
:100E7000B000B1018A012421A9016A08A400A501DA
:100E8000CD30B000B1018A012421A9016908A40074
:100E9000A501CD30B000B1018A012421A901650866
:100EA000A400A501CD30B000B1018A012421A9011F
:100EB0006408A400A501CD30B000B1018A0124214D
:100EC000A9016808A400A501CD30B000B1018A01D4
:100ED0002421A9016708A400A501CD30B000B1010B
:100EE0008A012421A9017B08A400A501CD30B0000E
:100EF000B1018A012421A9017A08A400A501CD30FD
:100F0000B000B1018A012421A9017D08A400A50136
:100F1000CD30B000B1018A012421A9017C08A400D0
:100F2000A501CD30B000B1018A0124212C308A0105
:100F3000CE200330A9006208A400A501CD30B00086
:100F4000B1018A0124212C308A01CE200330A9006E
:100F50006308A400A501CD30B000B1018A012421AD
:100F60000D308A01CE200D308A01CE200800463097
:100F70008A01032061308A01032069308A0103203D
:100F80006C308A01032020308A01032049308A0115
:100F9000032032308A01032043308A0103200D30C0
:100FA0008A0103200A308A010320080052308A0196
:100FB000032065308A01032061308A0103206430F8
:100FC0008A01032020308A01032052308A01032045
:100FD00054308A01032043308A0103200D308A01F6
:100FE00003200A308A0103200730B6000830B4001D
:100FF0000730B7000430B500D0308A0138208A119C
:101000000318B72F00308A0138208A110318B72F30
:101010008A011F208A110318B72FF0008A011F20B0
:101020008A110318B72FEE008A011F208A110318B6
:10103000B72FED008A011F208A110318B72FF10086
:101040008A011F208A110318B72FEC008A011F2084
:101050008A110318B72FEF008A011F208A11031885
:10106000B72FF2008A011D208A110318B72FEB0059
:101070000F307005FC0070307005FD007D08A00089
:10108000A10104308A017E21FD000F306E05FA00B7
:1010900070306E05FB007B08A000A10104308A01BE
:1010A0007E21FB000F306D05E70030306D05E80054
:1010B0006808A000A10104308A017E21E8000F30F9
:1010C0006C05E40030306C05E5006508A000A10166
:1010D00004308A017E21E5000F306F05E9001030F1
:1010E0006F05EA006A08A000A10104308A017E2190
:1010F000EA000F307205FF00F03072058316A00081
:1011000020088312A000A10104308A017E218316E9
:10111000A000831208004D308A0103204B308A0161
:10112000032020308A01032066308A0103206930C1
:101130008A0103206C308A01032065308A01032074
:1011400020308A0103206E308A01032061308A0139
:1011500003206D308A01032065308A01032020308E
:101160008A01032073308A01032074308A0103202E
:1011700072308A01032069308A0103206E308A01AF
:10118000032067308A0103200D308A0103200A30D2
:101190008A0103200730B6000830B4000730B700DA
:1011A0000430B500D0308A0138208A110318B72FD7
:1011B00000308A0138208A110318B72F8A011F20B6
:1011C0008A110318B72FF0008A011F208A11031813
:1011D000B72FEE008A011F208A110318B72FED00E8
:1011E0008A011F208A110318B72FF1008A011F20DE
:1011F0008A110318B72FEC008A011F208A110318E7
:10120000B72FEF008A011F208A110318B72FF200B1
:101210008A011D208A110318B72FEB000F306D05CE
:10122000E7006708D90030306D05E8006808A000C5
:10123000A10104308A017E21E8006808D8000F303F
:101240006C05E4006408D70030306C05E5006508E3
:10125000A000A10104308A017E21E5006508D600C6
:101260000F306F05E9006908D50010306F05EA00FE
:101270006A08A000A10104308A017E21EA006A0800
:10128000D4000F307205FF007F08D300F0307205E4
:101290008316A00020088312A000A10104308A0157
:1012A0007E218316A00020088312D20008004F3050
:1012B0008A01032070308A01032065308A010320EF
:1012C0006E308A01032020308A01032066308A01B3
:1012D000032069308A0103206C308A0103206530C5
:1012E0008A01032020308A010320A9015208A400AA
:1012F000A5010230B000B1018A012421A9015308DF
:10130000A400A5010230B000B1018A012421A90185
:101310005408A400A5010230B000B1018A012421C3
:10132000A9015508A400A5010230B000B1018A014D
:101330002421A9015608A400A5010230B000B10182
:101340008A012421A9015708A400A5010230B00098
:10135000B1018A012421A9015808A400A501023085
:10136000B000B1018A012421A9015908A400A501F6
:101370000230B000B1018A0124212E308A010320FD
:1013800063308A01032073308A01032076308A019A
:1013900003200D308A0103200A308A010320073020
:1013A000B6001030B4005430AA00AB01AE01AF015A
:1013B0004F308A01CE2050308A01CE2057308A012A
:1013C000CE2020308A01CE20A9015208A400A50118
:1013D000CD30B000B1018A012421A9015308A40035
:1013E000A501CD30B000B1018A012421A901540822
:1013F000A400A501CD30B000B1018A012421A901CA
:101400005508A400A501CD30B000B1018A01242106
:10141000A9015608A400A501CD30B000B1018A0190
:101420002421A9015708A400A501CD30B000B101C5
:101430008A012421A9015808A400A501CD30B000DB
:10144000B1018A012421A9015908A400A501CD30C8
:10145000B000B1018A0124212E308A01CE206330F0
:101460008A01CE2073308A01CE2076308A01CE20C8
:101470000D308A01CE20080043308A0103206C30F1
:101480008A0103206F308A01032073308A01032010
:1014900065308A01032020308A01032066308A01EA
:1014A000032069308A0103206C308A0103206530F3
:1014B0008A01032020308A010320A9015208A400D8
:1014C000A5010230B000B1018A012421A90153080D
:1014D000A400A5010230B000B1018A012421A901B4
:1014E0005408A400A5010230B000B1018A012421F2
:1014F000A9015508A400A5010230B000B1018A017C
:101500002421A9015608A400A5010230B000B101B0
:101510008A012421A9015708A400A5010230B000C6
:10152000B1018A012421A9015808A400A5010230B3
:10153000B000B1018A012421A9015908A400A50124
:101540000230B000B1018A0124212E308A0103202B
:1015500063308A01032073308A01032076308A01C8
:1015600003200D308A0103200A308A01032007304E
:10157000B6001030B4005430AA00AB01AE01AF0188
:1015800043308A01CE204C308A01CE2046308A0179
:10159000CE2020308A01CE20A9015208A400A50146
:1015A000CD30B000B1018A012421A9015308A40063
:1015B000A501CD30B000B1018A012421A901540850
:1015C000A400A501CD30B000B1018A012421A901F8
:1015D0005508A400A501CD30B000B1018A01242135
:1015E000A9015608A400A501CD30B000B1018A01BF
:1015F0002421A9015708A400A501CD30B000B101F4
:101600008A012421A9015808A400A501CD30B00009
:10161000B1018A012421A9015908A400A501CD30F6
:10162000B000B1018A0124212E308A01CE2063301E
:101630008A01CE2073308A01CE2076308A01CE20F6
:101640000D308A01CE2008000A308A0103200A30BA
:101650008A01032062308A01032061308A0103205D
:1016600064308A0103205F308A01032064308A01DC
:10167000032061308A01032074308A010320613025
:101680008A01032063008A15422B49308A01032016
:1016900044308A01032020308A01032065308A010A
:1016A000032072308A01032072308A0103206F30D8
:1016B0008A01032072308A0103200D308A01032041
:1016C0000A308A01032064008A15632B44308A01A2
:1016D00003204F308A0103204E308A010320453019
:1016E0008A0103200D308A0103200A308A01032079
:0E16F000051283160512640083128A157B2BE7
:02400E00FC3F75
:00000001FF
